:100000000C94F30A0C9415110C94EA100C94BF1084
:100010000C944A100C94D50F0C94600F0C94EB0EBA
:100020000C9401150C941D0B0C941D0B0C941D0BC2
:100030000C94AD270C9424280C9462270C941D0B6F
:100040000C941D0B0C941D0B0C9460740C941D0BE4
:100050000C942C270C9402270C941D0B0C941D0B54
:100060000C941D0B0C941D0B0C943D720C941D0BE9
:100070000C94CC260C94A2260C941D0B0C941D0BF6
:100080000C941D0B0C941D0B0C941D0BFD71007238
:10009000F371F77117721772047208720E7212728E
:1000A00008000000BE922449123EABAAAA2ABECD87
:1000B000CCCC4C3E00000080BEABAAAAAA3E0000F9
:1000C0000000BF000000803F0000000000084178F1
:1000D000D3BB4387D1133D190E3CC3BD4282AD2B28
:1000E0003E68EC8276BED98FE1A93E4C80EFFFBE20
:1000F00001C4FF7F3F000000000000407A10F35A67
:1001000000A0724E18090010A5D4E80000E8764857
:10011000170000E40B54020000CA9A3B000000E103
:10012000F505000080969800000040420F00000096
:10013000A08601000000102700000000E803000076
:1001400000006400000000000A0000000000010040
:10015000000000002C76D888DC674F0823DFC1DF61
:10016000AE59E1B1B796E5E3E453C63AE651997664
:1001700096E8E6C28426EB898C9B62ED407C6FFC9E
:10018000EFBC9C9F40F2BAA56FA5F490055A2AF7E0
:100190005C936B6CF9676DC11BFCE0E40D47FEF5E9
:1001A00020E6B500D0ED902E030094357705008051
:1001B000841E080000204E0A000000C80C333333B0
:1001C000330F986E12831141EF8D2114893BE65550
:1001D00016CFFEE6DB18D1844B381BF77C1D901D33
:1001E000A4BBE424203284725E228100C9F124EC95
:1001F000A1E53D270A4C6F676765723A7365744CD9
:100200006F676765724964206572726F72202D2076
:100210006578706563746564204E554C4C2070742D
:1002200072000A0D2020204C6F676765723A736573
:10023000744C6F67676572496420746F6F206C6FD0
:100240006E673A205472696D6D656420746F20008A
:100250002020204C6F633D006261747465727920C8
:10026000747970653D006D696E757465732C2054EA
:100270007A3D005D0A0D2020206C6F6767696E670C
:1002800020696E74657276616C3D0046726F6D20F8
:10029000656570726F6D20636F6D6D6F6E3A204C87
:1002A0006F676765722046696C65204E616D655B9E
:1002B00000466163746F72792064656661756C7461
:1002C000006D734C6F673031005D005D20736E5BB5
:1002D000005D20207265765B0046726F6D2065655B
:1002E00070726F6D20626F6F74204E616D655B0080
:1002F000302E3562004D313233343536373839617E
:100300006263646566676800656E7669726F44490A
:1003100059206D6179666C7900506172736520694E
:100320006E693B204E6F2066696C652000436F6DDF
:10033000706C657465642E004572726F72206F6E0A
:10034000206C696E65203A00506172736520696E99
:10035000693B200056005620474F4F443D00562031
:100360004D454449554D3D0056204C4F573D0020CA
:100370005468726573686F6C6473205553454142CD
:100380004C453D0042617474657279205479706502
:100390003D007365636F6E6473206F66204E495332
:1003A000542E00496E7465726E616C20436C6F63ED
:1003B0006B2077697468696E2000496E7465726E8F
:1003C000616C20436C6F636B207365742000426125
:1003D000642074696D657374616D702C206E6F7428
:1003E0002073657474696E6720636C6F636B2E0095
:1003F00050757474696E67206D6F64656D20746FDD
:1004000020736C65657000436F756C64206E6F744B
:100410002077616B65206D6F64656D20666F72205B
:10042000636C6F636B2073796E632E00436F756C22
:1004300064206E6F7420636F6E6E65637420746FDA
:1004400020696E7465726E657420666F7220636CCD
:100450006F636B2073796E632E0054686973206D2F
:1004600061792074616B6520757020746F207477DA
:100470006F206D696E757465732100417474656DCC
:100480007074696E6720746F20636F6E6E6563743D
:1004900020746F2074686520696E7465726E65746F
:1004A00020616E642073796E6368726F6E697A651D
:1004B000205254432077697468204E4953540044B5
:1004C0006174612077696C6C206265207361766568
:1004D0006420617300556E61626C6520746F2063E7
:1004E000726561746520612066696C6520746F2097
:1004F00073617665206461746120746F21005365B7
:100500007474696E672075702066696C65206F6E03
:1005100020534420636172640053657474696E678C
:100520002075702073656E736F72732E2E2E0054BB
:10053000696D65200053796E632077697468204E79
:10054000495354206F7665722057694669206E655D
:1005500074776F726B20000A0A2D2D2D70617273F3
:1005600065496E6920636F6D706C65746520002D40
:100570002D2D7061727365496E692000476F6F643D
:1005800020426174563D002D2D2D2D57616B6575F0
:1005900070003A20426174746572794C6F772D5304
:1005A0006C65657036307365632C20426174563D0E
:1005B0000054696E7947534D204C696272617279BB
:1005C0002076657273696F6E20004D6F64756C6183
:1005D0007253656E736F72732076657273696F6E96
:1005E00020000A2D2D2D426F6F742E204275696CEC
:1005F000643A20002D2D2D4E657752656164696E39
:10060000672043414E43454C4C45442D2D4C62617F
:1006100074745F563D00207374617475733D0043BC
:100620006F6C6C6563742072656164696E677320BA
:1006300026206C6F672E2062617474657279563D56
:10064000004552524F52004C4100544D00544D3021
:1006500000544D00414D3000465200414D310041A3
:10066000503000414D30004149002B2B2B004D599B
:10067000000054500027206661696C65642E0058A4
:10068000626565202700586265655769666920695B
:100690006E6974207465737420504153534544004F
:1006A000586265655769666920696E69742074656A
:1006B0007374204641494C4544202D20686F706575
:1006C00020697420776F726B73206E657874207464
:1006D000696D65004E53005D005862656557694657
:1006E0006920495023205B00586265655769466957
:1006F000206E6F7420726563656976656420495069
:1007000023202D686F706520697420776F726B737A
:10071000206E6578742074696D65004D59005862CB
:10072000656557694669206E6F7420415020526597
:100730006769737465726564202D2061626F7274DD
:10074000696E6720617474656D70742C20686F70B9
:100750006520697420776F726B73206E65787420E2
:1007600074696D65004149004C6F6F703D5365635E
:100770005D207278206462203A205374617475732E
:100780002023506F6C6C6564205374617475732002
:10079000657665727920317365632F3330736563D5
:1007A00000544D00534F00534D0049500044390050
:1007B0004438005052002700586265655769466901
:1007C00020496E697469616C697A696E6720496E47
:1007D0007465726E657420636F6D6D7320776974D4
:1007E00068206D6F64656D2027004C4174696D65EC
:1007F0002E6E6973742E676F76002D2D20526573EF
:10080000706F6E736520436F6465202D2D000A2084
:100810002D2D20556E61626C6520746F20457374B8
:1008200061626C69736820436F6E6E656374696F93
:100830006E20746F20456E7669726F44495920446A
:1008400061746120506F7274616C202D2D004932EB
:10085000435F3078363800616E6C674563205072B4
:100860006F6320446174612F507772004552524F7C
:100870005221204E6F2077656220636C69656E742B
:100880002061737369676E656420746F2070756290
:100890006C697368206461746121004143005752A0
:1008A00000434E004853004853000A4C6F67676589
:1008B000724D6F64656D3A3A73657457694669495C
:1008C00064206572726F72202D6E6F20627566668D
:1008D000657220000A4C6F676765724D6F64656DC5
:1008E0003A3A736574576946694964206572726F54
:1008F00072202D206578706563746564204E554CB8
:100900004C20707472000A0D2020204C6F676765C0
:10091000724D6F64656D3A736574576946694964D1
:1009200020746F6F206C6F6E673A205472696D6D22
:10093000656420746F20000A4C6F676765724D6FA5
:1009400064656D3A3A7365745769466950776420F7
:100950006572726F72202D6E6F20627566666572A9
:1009600020000A4C6F676765724D6F64656D3A3A97
:1009700073657457694669507764206572726F7247
:10098000202D206578706563746564204E554C4C4D
:1009900020707472000A0D2020204C6F676765720A
:1009A0004D6F64656D3A7365745769466950776435
:1009B00020746F6F206C6F6E673A205472696D6D92
:1009C000656420746F20003D005D20004E6F742030
:1009D000737570706F72746564205B004143544995
:1009E0004F4E2057726974652061626F727465643E
:1009F0002E20696E737472756374696F6E202700A0
:100A0000414354494F4E20434F5059206E6F74203C
:100A1000737570706F72746564207965743A004301
:100A20004F505900454550524F4D205772697465DB
:100A30002066696E697368656400414354494F4E8E
:100A40002057726974652061707020454550524F7F
:100A50004D20737461727465643A0057524954456D
:100A600000414354494F4E00555345520020746F86
:100A70002000424F4F54207462642000454550527C
:100A80004F4D2057726974652061626F727465649E
:100A90002E20696E737472756374696F6E202700FF
:100AA000454550524F4D2057726974652066696EF6
:100AB000697368656400454550524F4D205772690F
:100AC000746520737461727465643A00594553000B
:100AD000454550524F4D5F575249544500426F6152
:100AE0007264205265763A00424F4152445F52454B
:100AF0005600426F6172642053657269616C4E7575
:100B00006D203A00424F4152445F534E00426F61A4
:100B10007264204E616D653A00424F4152445F4E0F
:100B2000414D4500424F4F540020746F20004E4508
:100B300054574F524B20746264200027206E6F7709
:100B40002027004E4554574F524B20576946695055
:100B500077643A2077617320270057694669507798
:100B6000640027206E6F772027004E4554574F5260
:100B70004B205769466949643A2077617320270002
:100B8000576946694964004E4554574F524B0020FF
:100B9000746F200053454E534F52532074626420AB
:100BA0000053454E534F52530020746F2000434F63
:100BB0004D4D4F4E20746264200047454F475241CF
:100BC00050484943414C5F49443A0047454F4752DA
:100BD0004150484943414C5F494400434F4D4D4FBC
:100BE0004E205365742054696D655A6F6E6520659B
:100BF00072726F723B202872616E6765202D3132F0
:100C0000203A202B31322920726561643A00434F2B
:100C10004D4D4F4E205365742054696D655A6F6E6B
:100C200065203B200054494D455F5A4F4E450020FA
:100C3000536574204C69496F6E2054797065206546
:100C400072726F723B202872616E676520302D32A0
:100C50002920726561643A00434F4D4D4F4E204C40
:100C600069496F6E20547970653A20004C49494FAC
:100C70004E5F545950450020536574204C69496FAC
:100C80006E2054797065206572726F723B202872F5
:100C9000616E676520302D322920726561643A00EB
:100CA000434F4D4D4F4E204261747465727920540C
:100CB0007970653A2000424154544552595F545965
:100CC00050450029207769746820726561643A0094
:100CD0002053657420696E74657276616C2065724C
:100CE000726F72202872616E67653A20312D00287C
:100CF0006D696E292066726F6D2064656661756C22
:100D0000742000434F4D4D4F4E204C4F4747494EA6
:100D1000475F494E54455256414C5F4D494E5554DC
:100D200045532073657420746F3A20002055736911
:100D30006E67204D61782E2052656164696E672070
:100D400069676E6F7265642000434F4D4D4F4E20B2
:100D50004C4F4747494E475F494E54455256414CC8
:100D60005F4D494E55544553206D7573742062652F
:100D7000206C657373207468616E203A20004C4FBC
:100D80004747494E475F494E54455256414C5F4D87
:100D9000494E5554455300434F4D4D4F4E204C6FD7
:100DA000676765724964205365743A20004C4F4769
:100DB0004745525F494400434F4D4D4F4E007D2003
:100DC00055554944206E6F7420737570706F72743E
:100DD0006564007D206F7574206F662072616E6798
:100DE000652E204E6F7475736564007D007D2072E2
:100DF00065706C6163696E67207B00696E646578FD
:100E0000007D206D61746368202026206164646524
:100E1000642E003D7B000055554944730050524FED
:100E20005649444552206E6F7420737570706F720E
:100E30007465643A0050524F5649444552205365F8
:100E40007474696E672053616D706C696E67466576
:100E500061747572653A200053414D504C494E47BC
:100E60005F464541545552450050524F56494445FE
:100E7000522053657474696E6720636C6F756449A2
:100E8000643A2000434C4F55445F49440050524F50
:100E900056494445522053657474696E67207265E3
:100EA00067697374726174696F6E20746F6B656EBD
:100EB0003A2000524547495354524154494F4E5FDE
:100EC000544F4B454E0050524F5649444552002016
:100ED000002069732000207265706F7274732000A7
:100EE00020002069732063616C63756C61746564B4
:100EF00020746F20626520002D2D2D2D2D2D2D2D80
:100F00002D2D2D2D2D2D2D2D2D2D2D2D2D2D2D2D11
:100F10002D2D2D2D2D2D2D2D2D2D2D2D2D2D2D2D01
:100F20002D2D0045786974696E6720746573746946
:100F30006E67206D6F6465002D2D2D2D2D2D2D2DAF
:100F40002D2D2D2D2D2D2D2D2D2D2D2D2D2D2D00FE
:100F50002D2D2D2D2D2D2D2D2D2D2D2D2D2D2D2DC1
:100F60002D2D2D2D2D2D2D0043757272656E742043
:100F70006C6F676765722074696D65206973002DF9
:100F80002D2D2D2D2D2D2D2D2D2D2D2D2D2D2D2D91
:100F90002D2D2D2D2D2D2D2D2D2D2D2D2D2D2D2D81
:100FA0002D2D2D2D2D2D2D2D2D00456E7465726945
:100FB0006E672073656E736F722074657374696EEB
:100FC00067206D6F6465002D2D2D2D2D2D2D2D2D60
:100FD0002D2D2D2D2D2D2D2D2D2D2D2D2D2D2D2D41
:100FE0002D2D2D2D2D2D2D2D2D2D2D2D2D2D2D2D31
:100FF0002D002D3E00416C6C207661726961626C3F
:1010000065205555494427732061707065617220D1
:10101000746F20626520636F72726563746C7920EF
:10102000666F726D65642E0A006861732061206EC0
:101030006F6E2D756E697175652055554944210097
:1010400068617320616E20696E76616C69642055F9
:1010500055494421004C6F6767657220706F727448
:10106000696F6E206F662073657475702066696E97
:1010700069736865642E0A0053616D706C696E67F0
:101080002066656174757265205555494420697301
:101090003A006172652063616C63756C61746564AC
:1010A0002E0073656E736F727320616E6400636FE0
:1010B0006D652066726F6D007661726961626C6544
:1010C000732C206F662077686963680054686973C1
:1010D000206C6F676765722068617320612076619C
:1010E000726961626C6520617272617920776974DE
:1010F000680043757272656E74205254432074699F
:101100006D652069733A0027002720736E3A270027
:10111000207265763A2700426F6172643A2000209F
:101120004D6F64756C617253656E736F7273207668
:1011300065727320005377204275696C643A200011
:10114000202042617474657279547970653A200088
:1011500020547A3A200020204C6F6767696E6749F7
:101160006E74657276616C20286D696E293A200074
:101170004C6F636174696F6E3A200044617465203E
:10118000616E642054696D6520696E20555443007A
:10119000526573756C7420555549443A0052657315
:1011A000756C7420556E69743A005661726961629B
:1011B0006C65204E616D653A0053656E736F7220E9
:1011C0004E616D653A0053616D706C696E672046C3
:1011D00065617475726520555549443A2000446133
:1011E0007461204C6F676765722046696C653A20B0
:1011F0000044617461204C6F676765723A20004457
:101200006174612077696C6C206E6F742062652058
:1012100073617665642100536C6176652F4368695C
:10122000702073656C6563742070696E20666F72E0
:10123000205344206361726420686173206E6F7470
:10124000206265656E207365742E004461746120B0
:1012500077696C6C206E6F742062652073617665AF
:101260006421004572726F723A20534420636172A8
:1012700064206661696C656420746F20696E6974AE
:1012800069616C697A65206F72206973206D69737A
:1012900073696E672E001F1C1F1E1F1E1F1F1E1F3F
:1012A0001E1F494400454500504B004552524F52C5
:1012B0000D004F4B0D004545004442004C4D0025AC
:1012C0005600434900736574566172555549442070
:1012D0006572726F72202D206E6577206469646E6E
:1012E000277420776F726B20666F720050696E00F2
:1012F0002D2D2D2D2D205741524E494E47202D2D5D
:101300002D2D2D20212121212121212121212121AA
:101310002121212121212121004261642074696D54
:10132000652000212121212121212121212121218B
:1013300021212121212121202D2D2D2D2D2057410D
:10134000524E494E47202D2D2D2D2D20003A303064
:10135000003A3030003A3030003A303000455252D6
:101360004F52004F4400544D00544D00444500443A
:101370004C0049500043543634004754363400453D
:1013800052524F520D004F4B0D0041503000212161
:10139000212121212121212121212121212121213D
:1013A0002121202D2D2D2D2D205741524E494E47C4
:1013B000202D2D2D2D2D2000212121212121212104
:1013C0002121202D2D2D2D2D205741524E494E47A4
:1013D000202D2D2D2D2D20212121212121212121C3
:1013E00021002D2D2D2D2D205741524E494E4720A5
:1013F0002D2D2D2D2D2021212121212121212121A2
:1014000021212121212121212121005468652063EE
:10141000757272656E7420636C6F636B2074696D96
:10142000657374616D70206973206E6F74207661CE
:101430006C696421002121212121212121212121E7
:10144000212121212121212121202D2D2D2D2D2052
:101450005741524E494E47202D2D2D2D2D20002134
:10146000212121212121212121202D2D2D2D2D2032
:101470005741524E494E47202D2D2D2D2D202121F3
:101480002121212121212121002D2D2D2D2D2057FC
:1014900041524E494E47202D2D2D2D2D2021212109
:1014A000212121212121212121212121212121212C
:1014B00021002D2D2D2D5C2F000A205C2F2D2D2D90
:1014C0002D204C696E6520536176656420746F0031
:1014D000556E61626C6520746F2077726974652047
:1014E000746F205344206361726421002D2D2D2DD3
:1014F0002D2D2D2D2D2D2D2D2D2D2D2D2D2D2D2D1C
:101500002D2D2D2D2D2D2D2D2D2D2D2D2D2D2D2D0B
:101510002D2D2D2D2D2D0A002D2D2D2D2D2D2D2D4B
:101520002D2D2D2D2D2D2D2D2D2D2D2D2D2D2D2DEB
:101530002D2D2D2D2D2D2D2D2D2D2D2D2D2D2D2DDB
:101540002D2D0000002000230026002900000102AC
:101550000304050607000102030405060700010253
:10156000030405060700010203040506070404043A
:10157000040404040402020202020202020303033E
:10158000030303030301010101010101010102043D
:10159000081020408001020408102040800102044D
:1015A0000810204080010204081020408000002123
:1015B00000240027002A0000002200250028002B1C
:1015C00000000000000403080700000001020009F9
:1015D0000A00000000000000000000000000000001
:1015E0000000177CE58211241FBECFEFD0E4DEBFE0
:1015F000CDBF17E0A0E0B1E0E0EDFCE101E00BBF02
:1016000002C007900D92A633B107D9F724E1A6E3F3
:10161000B7E001C01D92AB3AB207E1F71AE0C2EFA2
:10162000DAE004C02197FE010E94368BC13FD1074A
:10163000C9F70E94AA740C945B8E0C940000DC0124
:10164000ED91FC910688F789E02D099591E08111D3
:1016500001C090E0892F08950F931F93CF93DF93DC
:1016600000D000D000D0CDB7DEB78C01DC01ED9109
:10167000FC910084F185E02D0995892BC9F41B822A
:101680001C821D821E82D8011C96ED91FC911D9733
:1016900045855685678570898B819C81AD81BE812A
:1016A000481759076A077B0729F0F801858903C0A5
:1016B00081E001C080E026960FB6F894DEBF0FBE31
:1016C000CDBFDF91CF911F910F910895DC011C9642
:1016D000ED91FC911D9780819181DC01ED91FC9150
:1016E0000680F781E02D0994DC011C96ED91FC91B8
:1016F0001D9780819181DC01ED91FC910484F58539
:10170000E02D0994CF93DF931F92CDB7DEB76983A5
:10171000DC01ED91FC910280F381E02D41E050E08D
:10172000BE016F5F7F4F09950F90DF91CF910895B4
:101730000F931F93CF93DF9300D000D000D0CDB78D
:10174000DEB7DC01ED91FC91048CF58DE02D2AEDE6
:1017500032E03A832983DB0112960D911D912D9180
:101760003C9115970B831C832D833E8320E030E052
:10177000BE016F5F7F4F099526960FB6F894DEBFC6
:101780000FBECDBFDF91CF911F910F910895DC0166
:10179000ED91FC91028CF38DE02D2BE430E0099467
:1017A000809141108111FCCF0895809145108F5F89
:1017B000843408F080E0909144109817E1F32FB73B
:1017C000F89490914110992341F0E82FF0E0E55012
:1017D000F04F6083809345101DC081E080934110DD
:1017E0006093401010923F1082E086BB80916F00A2
:1017F000826080936F00809180008F7B80688093EF
:10180000800080918400909185004096909389009B
:10181000809388002FBF81E090E00895FC018485CB
:1018200083FF0DC084A195A1A6A1B7A1448D558DBC
:10183000668D778D841B950BA60BB70B03C080E0DC
:1018400090E0DC01811520E89207A105B10520F0A8
:101850008FEF9FE7A0E0B0E0089580E090E008956A
:10186000CF93DF93EC0162E070E080E090E00E94B3
:101870001A74EC85FD8580819181DC01ED91FC91EC
:101880000284F385E02DDF91CF910994CF93DF930C
:10189000EC0162E070E080E090E00E941A74EC8558
:1018A000FD8580819181DC01ED91FC910084F185C1
:1018B000E02DDF91CF910994CF92DF92EF92FF92CA
:1018C0000F931F93CF93DF938C01D62FC72F6A01FD
:1018D00062E070E080E090E00E941A74D8011C96EB
:1018E000ED91FC911D97E080F1800D2F1C2FC0E041
:1018F000D0E0CC16DD0651F0C7010E94642597FDAB
:1019000005C0F80181938F012196F3CFCE01DF91BD
:10191000CF911F910F91FF90EF90DF90CF9008959E
:10192000EF92FF920F931F93CF93DF93EC018B0104
:101930007A0162E070E080E090E00E941A74A701F2
:10194000B8018C859D85DF91CF911F910F91FF90FC
:10195000EF900C940464CF92DF92EF92FF920F937A
:101960001F93CF93DF9300D000D000D0CDB7DEB768
:101970008C016B017A01FC01848595850E94CC3332
:10198000F80126858AED92E09A838983F6018281A7
:101990009381A481B5818B839C83AD83BE83A70192
:1019A000BE016F5F7F4FF801848595850E941D61A0
:1019B000F801858B90E026960FB6F894DEBF0FBE37
:1019C000CDBFDF91CF911F910F91FF90EF90DF90EE
:1019D000CF9008950C960C9425488F929F92AF92C9
:1019E000BF92CF92DF92EF92FF920F931F93CF930C
:1019F000DF931F92CDB7DEB78C01FC01848C958CF0
:101A0000A68CB78CC08CD18CE28CF38CBE016F5F3E
:101A10007F4F0C960E944C47019719F4898190E002
:101A200002C08FEF9FEF8F3FFFEF9F0749F0F80154
:101A3000848E958EA68EB78EC08ED18EE28EF38E5A
:101A40000F90DF91CF911F910F91FF90EF90DF905A
:101A5000CF90BF90AF909F908F900895CF93DF93DA
:101A60001F92CDB7DEB7BE016F5F7F4F0C960E940D
:101A70004C47019719F4898190E002C08FEF9FEFE6
:101A80000F90DF91CF9108950C960C940D5A8F9280
:101A90009F92AF92BF92DF92EF92FF920F931F93AC
:101AA000CF93DF93EC01D62E1BA1112391F00E945E
:101AB00054748CA09DA0AEA0BFA0DC01CB018819FE
:101AC0009909AA09BB0980319742A105B10508F41B
:101AD00054C0CE010E94CC3384E0F82EE12CDE14F9
:101AE00009F44AC06E817F81665F7F4F072E000C2C
:101AF000880B990B0E941A746AE676E088819981B6
:101B00000E946C264E815F81440F551F052E000CEC
:101B1000660B770B0FE713E126E833E1CE010E9455
:101B2000094C182F81111BC0FA94F11018C08A8536
:101B300087FD0DC060E00E94987361E070E080E076
:101B400090E00E941A7461E08A850E9498736AEF9F
:101B500070E080E090E00E941A7494E0F92EE39423
:101B6000113009F0BCCF1BA30E9454746CA37DA359
:101B70008EA39FA311E001C010E0812FDF91CF91D0
:101B80001F910F91FF90EF90DF90BF90AF909F90CB
:101B90008F9008958F929F92AF92BF92FF920F9372
:101BA0001F93CF93DF93EC01FBA0FF2021F08BA1CB
:101BB000882331F008C065E00E94470D8111F7CFFE
:101BC00084E090E0FEC088859985892B19F4CE01C8
:101BD0000E94C62967E676E0CE010E94E13440E12A
:101BE00057E260E070E0CE010E94772928853985B0
:101BF0002130364009F0A8C08332910509F4D7C0DE
:101C00005CF4833091052CF4813091050CF4A6C06E
:101C1000B9C0439789F0C9C0833491050CF0AFC0B7
:101C2000803491050CF0AEC08432910509F4ACC04B
:101C3000879709F4A9C0B9C065E0CE010E94470D9D
:101C4000882309F4B4C088859985892B19F4CE01BD
:101C50000E94C6298885998581309640B9F06BE548
:101C600076E0CE010E94E1344FE753E166E873E18C
:101C7000CE010E944B4C813021F0CE010E944129BF
:101C800096C0CE010E9453298823B9F368E576E017
:101C9000CE010E94E1344FE753E166E873E1CE01E3
:101CA0000E944B4C813049F71BA288859985813071
:101CB000964029F460ED77E080E090E004C064E6AF
:101CC00070E080E090E00E941A740E9454744B010E
:101CD0005C010E945474DC01CB0188199909AA099E
:101CE000BB0980369A4EA105B10568F461E0CE01CA
:101CF0000E94470D811107C06AEF70E080E090E01C
:101D00000E941A74E6CF8885998581309640A9F0A3
:101D100064E576E0CE010E94E1344FE753E166E8E6
:101D200073E1CE010E944B4C813009F0A6CFCE0169
:101D30000E945329882309F4A0CFCE010E94412993
:101D4000CE010E94CA5F33C085329105E9F04CF4A0
:101D50008432910554F582329105A4F4892B49F11E
:101D600024C08D32910544F48B329105F4F48A97A6
:101D7000E1F463E676E00CC08F32910539F08F3FD5
:101D8000910599F402E016C003E014C06FE576E017
:101D9000CE010E94E1344FE753E166E873E1CE01E2
:101DA0000E944B4CCE010E94532904E003C001E085
:101DB00001C000E010E0F11003C0CE010E944129F3
:101DC000C801DF91CF911F910F91FF90BF90AF900D
:101DD0009F908F9008951F920F920FB60F9211242B
:101DE0000BB60F922F933F934F935F936F937F9315
:101DF0008F939F93AF93BF93CF93EF93FF9329B1AB
:101E0000C0919D138091E5139091E113322F30958D
:101E100093238223892B90917300C227C923C8235F
:101E200020939D13CC23C1F1C0FF05C0E0919E1308
:101E3000F0919F130995C1FF05C0E091A013F091A7
:101E4000A1130995C2FF05C0E091A213F091A3135D
:101E50000995C3FF05C0E091A413F091A51309955E
:101E6000C4FF05C0E091A613F091A7130995C5FF23
:101E700005C0E091A813F091A9130995C6FF05C00C
:101E8000E091AA13F091AB130995C7FF05C0E0914B
:101E9000AC13F091AD130995FF91EF91CF91BF91E4
:101EA000AF919F918F917F916F915F914F913F91F2
:101EB0002F910F900BBE0F900FBE0F901F90189593
:101EC0001F920F920FB60F9211240BB60F922F9301
:101ED0003F934F935F936F937F938F939F93AF93B2
:101EE000BF93CF93EF93FF9326B1C091AE13809130
:101EF000E6139091E213322F309593238223892B9E
:101F000090916D00C227C923C8232093AE13CC2320
:101F1000C1F1C0FF05C0E091AF13F091B013099576
:101F2000C1FF05C0E091B113F091B2130995C2FF52
:101F300005C0E091B313F091B4130995C3FF05C038
:101F4000E091B513F091B6130995C4FF05C0E09177
:101F5000B713F091B8130995C5FF05C0E091B91307
:101F6000F091BA130995C6FF05C0E091BB13F0913B
:101F7000BC130995C7FF05C0E091BD13F091BE13D6
:101F80000995FF91EF91CF91BF91AF919F918F9163
:101F90007F916F915F914F913F912F910F900BBE69
:101FA0000F900FBE0F901F9018951F920F920FB6B3
:101FB0000F9211240BB60F922F933F934F935F9381
:101FC0006F937F938F939F93AF93BF93CF93EF9331
:101FD000FF9323B1C091BF138091E7139091E31356
:101FE000322F309593238223892B90916C00C22746
:101FF000C923C8232093BF13CC23C1F1C0FF05C060
:10200000E091C013F091C1130995C1FF05C0E091A3
:10201000C213F091C3130995C2FF05C0E091C41328
:10202000F091C5130995C3FF05C0E091C613F09167
:10203000C7130995C4FF05C0E091C813F091C913F7
:102040000995C5FF05C0E091CA13F091CB1309951E
:10205000C6FF05C0E091CC13F091CD130995C7FFE1
:1020600005C0E091CE13F091CF130995FF91EF9148
:10207000CF91BF91AF919F918F917F916F915F9120
:102080004F913F912F910F900BBE0F900FBE0F906D
:102090001F9018951F920F920FB60F9211240BB636
:1020A0000F922F933F934F935F936F937F938F93F1
:1020B0009F93AF93BF93CF93EF93FF9320B1C091C2
:1020C000D0138091E8139091E413322F309593232D
:1020D0008223892B90916B00C227C923C8232093A8
:1020E000D013CC23C1F1C0FF05C0E091D113F09112
:1020F000D2130995C1FF05C0E091D313F091D41319
:102100000995C2FF05C0E091D513F091D61309954A
:10211000C3FF05C0E091D713F091D8130995C4FF10
:1021200005C0E091D913F091DA130995C5FF05C0F8
:10213000E091DB13F091DC130995C6FF05C0E09137
:10214000DD13F091DE130995C7FF05C0E091DF13A1
:10215000F091E0130995FF91EF91CF91BF91AF916D
:102160009F918F917F916F915F914F913F912F91AF
:102170000F900BBE0F900FBE0F901F9018951F92DF
:102180000F920FB60F9211240BB60F922F933F931D
:102190004F935F936F937F938F939F93AF93BF936F
:1021A000EF93FF93E0919B13F0919C130995FF919E
:1021B000EF91BF91AF919F918F917F916F915F91BF
:1021C0004F913F912F910F900BBE0F900FBE0F902C
:1021D0001F9018951F920F920FB60F9211240BB6F5
:1021E0000F922F933F934F935F936F937F938F93B0
:1021F0009F93AF93BF93EF93FF93E0919913F09167
:102200009A130995FF91EF91BF91AF919F918F9193
:102210007F916F915F914F913F912F910F900BBEE6
:102220000F900FBE0F901F9018951F920F920FB630
:102230000F9211240BB60F922F933F934F935F93FE
:102240006F937F938F939F93AF93BF93EF93FF937E
:10225000E0919713F09198130995FF91EF91BF9139
:10226000AF919F918F917F916F915F914F913F912E
:102270002F910F900BBE0F900FBE0F901F901895CF
:10228000BF92CF92DF92EF92FF920F931F93CF9363
:10229000DF93CDB7DEB72C970FB6F894DEBF0FBE35
:1022A000CDBF6C01FC01848595850E94CC33F6017D
:1022B000E484F584C7010E94CC33F701178E10A285
:1022C00011A212A2B3A0BB2041F161E576E0C701E3
:1022D0000E94E13428E833E140E050E0B701CE014C
:1022E00007960E94F728F7018085918581309640F6
:1022F000D9F46DE476E0C7010E94E1340FE713E101
:1023000026E833E148E853E160E070E0C7010E944D
:10231000094CC7010E94532907C065E0C7010E940C
:10232000470D8111D2CF2AC0BE01695F7F4FCE0118
:1023300001960E940125AE014F5F5F4F6AE476E08F
:10234000C7010E94AD60CE0101960E94C4240FE730
:1023500013E126E833E148E853E160E070E0C701AB
:102360000E94094CC7010E945329B11003C0C70144
:102370000E944129CE0107960E94C424F60184855B
:1023800095850E94CC33F601158A2C960FB6F894E9
:10239000DEBF0FBECDBFDF91CF911F910F91FF9098
:1023A000EF90DF90CF90BF9008952F923F924F9281
:1023B0005F926F927F928F929F92AF92BF92CF92D5
:1023C000DF92EF92FF920F931F93CF93DF93CDB7DE
:1023D000DEB762970FB6F894DEBF0FBECDBF9E8703
:1023E0008D876B015A8B498B3901DC011C968D91CD
:1023F0009C911D970E94CC33ED85FE85F685FF8765
:10240000AD85BE851C960D911C911D97F80133A0DA
:102410003320A9F0B601CE0101967C010E940A2565
:10242000580191E1A90EB11CB701C5010E943723E3
:10243000982EC7010E94C424911022C007C065E0F5
:10244000C8010E94470D8111E5CF09C1B601C7013E
:102450000E940A25EA14FB0421F0B701C5010E947D
:102460004823C7010E94C424D80159961C92599749
:102470005A961C925A975B961C925B975C961C929C
:102480001B821C821D821E82F801418D528D638D3C
:10249000748D8B819C81AD81BE81481759076A0775
:1024A0007B0709F0ABC060E176E0CE0107960E94A1
:1024B0000A2560E170E0CE0107960E9482230E9407
:1024C00054744B015C0128EE33E0D3010E943F8B32
:1024D0002B013C01D80193962C9021105DC065E042
:1024E000C8010E94470D811157C08AED92E09A837E
:1024F00089831B821C821D821E8273C00E945474B9
:10250000DC01CB0188199909AA09BB098415950535
:10251000A605B70590F462E070E080E090E00E94CC
:102520001A74F80180819181DC01ED91FC910084A5
:10253000F185E02D099504970CF3F8016081718114
:10254000C7010E94584CB701CE0107960E9448234C
:10255000C7010E94C424CE0107960E94A722CE0183
:1025600007960E94F746811111C061E476E0C70129
:102570000E94C924B701CE0107960E943723888B99
:10258000C7010E94C424B889BB23D9F064EC79E068
:1025900080E090E00E941A740E945474DC01CB0128
:1025A00088199909AA09BB0984159505A605B705D7
:1025B00008F073C0A60167E476E0C8010E946F349A
:1025C000B0CF211008C0DD24D394C8010E94412956
:1025D000DD2009F48ACFBE01695F7F4FC7010E94E9
:1025E000ED33CE0107960E94C4248B819C81AD817E
:1025F000BE81F801818F928FA38FB48FD801599635
:102600004D915D916D917C915C971B821C821D8226
:102610001E828B819C81AD81BE81481759076A0754
:102620007B07B1F08AED92E09A838983F801818D6E
:10263000928DA38DB48D8B839C83AD83BE832F85B8
:1026400049895A89B701C8010E941D61F82E01C04D
:10265000F12C311003C0C8010E9441298F2DAD8596
:10266000BE8555968C9390E062960FB6F894DEBFC7
:102670000FBECDBFDF91CF911F910F91FF90EF90D3
:10268000DF90CF90BF90AF909F908F907F906F9092
:102690005F904F903F902F900895211026CFD12C1E
:1026A00094CFCF93DF93E901FB011082FA011082EE
:1026B000C2960E94D3429983888381E0DF91CF91B3
:1026C0000895FC01838587FD05C0648591E0692735
:1026D0000E94987381E00895FC01838587FD03C003
:1026E00064850E94987381E008953F924F925F92B3
:1026F0006F927F928F929F92AF92BF92CF92DF9212
:10270000EF92FF920F931F93CF93DF93EC018AA177
:102710009BA1ACA1BDA1892B8A2B8B2B39F4E8811D
:10272000F9810084F185E02DCE010995E881F981D8
:1027300000A0F1A1E02DCE0109950E9454740AA1D8
:102740001BA12CA13DA1DC01CB01801B910BA20B95
:10275000B30B098D1A8D2B8D3C8D80179107A20725
:10276000B30758F3E881F98102A4F3A5E02DCE0167
:102770000995811107C0E881F98106A0F7A1E02D34
:10278000CE01099583E0382ECE01C2967C016E0100
:1027900095E5C90ED11C3A94332029F18D8C9E8C7D
:1027A000AF8CB8A0A4EF8A0EA1E09A1EA11CB11CA8
:1027B0000E9454742B013C010E945474DC01CB0133
:1027C00084199509A609B70988159905AA05BB05B5
:1027D00008F447C0E881F9810088F189E02DCE0135
:1027E00009958111D8CF10E08AA99BA9DC01ED9150
:1027F000FC910084F185E02D0995892B79F08AA957
:102800009BA9DC01ED91FC910284F385E02D0995F3
:1028100060E070E0CB010E941A74E6CF8AA58111B6
:1028200009C0E881F9810480F581E02DCE01099588
:10283000182F04C0C7010E94CA5F1823FE01E65A80
:10284000FF4FF586E4861686158AFDABECAB1123A7
:1028500009F44CC089A187FD49C061E00E949873CA
:1028600045C0F601808181110BC065E0C7010E945F
:10287000470D182F882389F1C7010E9441292DC0D7
:102880000EA91FA965E675E08AA99BA90E944A26A0
:10289000B8018AA99BA90E944A268AA99BA9DC01A2
:1028A000ED91FC910680F781E02D099560E070E0E4
:1028B000CB010E941A740BEA12E122EB32E148ECE0
:1028C00050E060E070E0C7010E94094C813021F0C7
:1028D000F601108210E001C011E06AEF70E080E0C4
:1028E00090E00E941A7411117FCF66CF812FDF9183
:1028F000CF911F910F91FF90EF90DF90CF90BF90FD
:10290000AF909F908F907F906F905F904F903F908F
:102910000895FF920F931F93CF93DF938C01FC01D7
:1029200085859685A785B089892B8A2B8B2B79F095
:10293000838187FD3EC00E946F7321E0892B09F4DB
:1029400020E081E0F8019481291352C054C0F801BD
:10295000C3850C2E000CDD0BFE01E357FA4EE4910B
:102960006E2F70E080E090E00E9462890E94718C7E
:10297000FE01E359FA4EE491F0E0EE0FFF1FED5B2C
:10298000FA4EA591B491CC91D0E028E132E741E331
:102990005FE30E94BC8B0E942E8C02C0D595C79528
:1029A0006A95E2F7C17081E0F8019485C91320C0EF
:1029B00022C085E0F82EE801E29661E776E0CE01DC
:1029C0000E94E1340BEA12E122EB32E144E650E0EE
:1029D00060E070E0CE010E94094C813059F062E362
:1029E00070E080E090E00E941A74FA94F110E5CF54
:1029F00080E001C081E0DF91CF911F910F91FF90A6
:102A000008951F920F920FB60F9211248F939F93E8
:102A1000AF93BF9380918F1390919013A0919113D6
:102A2000B09192130197A109B10980938F139093EC
:102A30009013A0939113B093921380918F13909160
:102A40009013A0919113B0919213892B8A2B8B2B09
:102A500051F414BE8091600088618093600088E02A
:102A60008093600001C0A895BF91AF919F918F9115
:102A70000F900FBE0F901F9018950FB6F894A89561
:102A800080916000886180936000109260000FBEAA
:102A90000895DC01F89414BEE0E6F0E090819861BE
:102AA000908381E6808378948D919D910D90BC9167
:102AB000A02D23E0B695A795979587952A95D1F7F0
:102AC00080938F1390939013A0939113B0939213CC
:102AD0000895CF93DF93EC018AEA92E0998388838B
:102AE000CE018D5B9F4F0E94C4248AE492E09983BB
:102AF0008883CE018C96DF91CF910C94C424CF9320
:102B0000DF93EC010E946915CE01DF91CF910C9407
:102B1000CA83CF92DF92EF92FF920F931F93CF93CE
:102B2000DF93CDB7DEB72C970FB6F894DEBF0FBE9C
:102B3000CDBF8C010E5C1F4F7C0125E5E20EF11C20
:102B4000F701D080DD2029F0F701F080F1101CC0E2
:102B50000EC065E0C8010E94470D8111F5CFC12C60
:102B60009CE3D92E9CE1E92E96ECF92E68C065E035
:102B7000C8010E94470D811107C060E176E0CE01D7
:102B800007960E940A2524C062E776E0C8010E94E9
:102B9000E13428EE33E040E050E0B801CE01019688
:102BA0000E94F728F11003C0C8010E94412918862D
:102BB0001F821A8619861C861B86BE016F5F7F4F97
:102BC000CE0107960E944823CE0101960E94C4249C
:102BD000CE0107960E94F746811126C0CE010196CC
:102BE0007C0185E0F70111928A95E9F745E050E014
:102BF000B701CE0107960E94554A40E150E060E0DF
:102C000070E0C7010E945384F62ED11003C0C801A2
:102C10000E9441296F2DFF0C770B880B990B0E94A6
:102C200064896B017C0107C0C12C8CE3D82E8CE138
:102C3000E82E86ECF82ECE0107960E94C424C70128
:102C4000B6012C960FB6F894DEBF0FBECDBFDF9154
:102C5000CF911F910F91FF90EF90DF90CF9008954B
:102C6000CF92DF92EF92FF920F931F93CF93DF9358
:102C7000CDB7DEB72C970FB6F894DEBF0FBECDBF31
:102C80008C010E94CA0D892B09F06DC0F801F3A0D8
:102C9000F1100DC065E0C8010E94470D811107C009
:102CA00060E176E0CE0101960E940A253FC06EE603
:102CB00076E0C8010E94E13460E176E0CE0107963B
:102CC0000E940A2560E170E0CE0107960E948223EF
:102CD00020E335E740E050E0B801CE0101960E94C4
:102CE000F728BE016F5F7F4FCE0107960E944823F1
:102CF000CE0101960E94C424F11003C0C8010E94B5
:102D00004129CE0107960E94A7221A8219821C82AD
:102D10001B821E821D82BE01695F7F4FCE0101961C
:102D20000E944823CE0107960E94C424BE016F5F13
:102D30007F4FCE0107960E94ED33C984DA84EB847D
:102D4000FC84CE0101960E94C4241B821C821D8239
:102D50001E824B815C816D817E8181E04C155D0519
:102D60006E057F0509F480E02C960FB6F894DEBF5F
:102D70000FBECDBFDF91CF911F910F91FF90EF90CC
:102D8000DF90CF900895C2960C9430164F925F92C8
:102D90006F927F928F929F92AF92BF92CF92DF926B
:102DA000EF92FF920F931F93CF938C012A013B0167
:102DB0007C0182E3E80EF11CC7010E943016C82F87
:102DC000882311F0C1E048C05801E7EBAE0EB11CFA
:102DD0006801F5EBCF0ED11CF50140815181F60160
:102DE00060817181C7010E945B438823A9F3F801C8
:102DF000EB5AFF4F1081112329F00E9454744B01AC
:102E00005C0112C065E0C7010E94470D8111F5CF3A
:102E100023C0C7010E94301681111AC06AEF70E00A
:102E200080E090E00E941A740E945474DC01CB018F
:102E300088199909AA09BB0984159505A605B7053E
:102E400040F3111109C0C0E0C7010E94412904C02C
:102E50001111B8CFC1E0F8CF8C2FCF911F910F91F6
:102E6000FF90EF90DF90CF90BF90AF909F908F90AA
:102E70007F906F905F904F9008952F923F924F9266
:102E80005F926F927F928F929F92AF92BF92CF92FA
:102E9000DF92EF92FF920F931F93CF93DF93CDB703
:102EA000DEB7C054D1090FB6F894DEBF0FBECDBF58
:102EB0007C016C0122E3C20ED11CC6010E94CA5FD4
:102EC000982EF701E65AFF4FD586C4861686158AD6
:102ED000D701D596FC93EE93D497DA966D917C91B9
:102EE000DB978E010F5F1F4FC8010E94061F57011D
:102EF000BCE2AB0EB11C0A151B0521F0B801C501DF
:102F00000E944823C8010E94C42465E0C6010E94B3
:102F1000470D882309F4FAC1C6010E94C629F701AA
:102F200062AD73ADC8010E94061F0A151B0521F092
:102F3000B801C5010E944823C8010E94C424B501FC
:102F4000C8010E94012546EB57E0B80188EB97E0E5
:102F50000E94EE45C8010E94C42448E655E063EB98
:102F600077E0C6010E946F344BEA52E162EB72E1F6
:102F7000C6010E944B4C41E050E060EB77E0C60197
:102F80000E94A8344BEA52E162EB72E1C6010E9452
:102F90004B4C41E050E06DEA77E0C6010E94A83456
:102FA0004BEA52E162EB72E1C6010E944B4C41E0F8
:102FB00050E06AEA77E0C6010E94A8344BEA52E189
:102FC00062EB72E1C6010E944B4C41E050E067EABF
:102FD00077E0C6010E94A8344BEA52E162EB72E14D
:102FE000C6010E944B4C48EC50E064EA77E0C60111
:102FF0000E94A8344BEA52E162EB72E1C6010E94E2
:103000004B4CF701E954FF4F408151813297608169
:103010007181C6010E945B4340E450E061EA77E0C1
:10302000C6010E94A8344BEA52E162EB72E1C6018C
:103030000E944B4C21968FAF2197C6010E945329C5
:103040008E010E5D1F4F60E176E0C8010E940A25E7
:1030500088E697E00E94AF280E9454741B012C015F
:10306000912C612C712C78010E945474DC01CB01ED
:1030700082199309A409B509803E9349A440B1057A
:1030800008F059C165E677E0C6010E94E13440E1ED
:1030900057E260E070E0C6010E947729882E1BAEDF
:1030A0001AAE1DAE1CAE1FAE1EAE40E1BE016F5F7C
:1030B0007F4F90E00E94E186BE016F5F7F4FCE019F
:1030C000CA960E94962460E070E0CE01C4960E94E9
:1030D00051600E9454741FA61EA619AA18AA1BAA02
:1030E0001AAA0E94628920E030E04AE754E40E9474
:1030F000BC8B8E010F5F1F4F22E044E00E941283C1
:10310000BC01CE018E960E94962419A618A61BA675
:103110001AA61DA61CA64AE0B801C3010E94E186BA
:10312000B801CE0188960E949624BE01685D7F4F4B
:10313000C8010E94012568E775E0C8010E94492482
:10314000BE01625D7F4F0E9462246DE675E00E94C1
:103150004924BE016C5C7F4F0E94622460E775E0E9
:103160000E944924BE01665C7F4F0E946224BC011C
:10317000C7010E94AD24C8010E94C424CE018896D4
:103180000E94C424CE018E960E94C424CE01C4960F
:103190000E94C424CE01CA960E94C424811037C064
:1031A00019A618A61BA61AA61DA61CA64AE0B801B9
:1031B000892D90E00E94E186B801CE0188960E9498
:1031C000962464E775E0C8010E940A25BE01685D87
:1031D0007F4FC8010E946224BC01C7010E944A605F
:1031E000C8010E94C424CE0188960E94C424B7015D
:1031F000C8010E940125B80180EC98E00E945A267F
:10320000C8010E94C424939423E02915D0F0B7018B
:10321000CE0101960E940125BE016F5F7F4F80ECB9
:1032200098E00E945A26CE0101960E94C42468EEBE
:1032300073E080E090E00E941A748FEF681A780AB9
:1032400013CF60E176E0CE0101960E940A2594EF4B
:10325000492E55245394612C712CC301B2010E9454
:103260001A746BE177E0C6010E94E1343BEAE32E79
:1032700032E1F32E02EB12E19E012F5F3F4F48EE49
:1032800053E060E070E0C6010E94E24A6AE775E040
:10329000CE0188960E940A25BE01685D7F4FCE014F
:1032A00001960E940723892B09F451C011E08D81FA
:1032B0009E81089708F44BC0CE0188960E94C424D2
:1032C000111147C060E176E0CE0101960E9496247C
:1032D000A4EF4A0EA1E05A1E611C711CB4E34B1608
:1032E000B1E25B066104710409F0B7CF88EE96E0A5
:1032F0000E94AF28912CCE0101960E94C424C601E1
:103300000E944129CE0182960E94C424911099C046
:10331000B501CE0101960E94012545E756E0BE01A8
:103320006F5F7F4F8FE796E00E94EE45CE010196DA
:103330000E94C42486C08EE197E00E94AF2864E614
:1033400070E080E090E00E941A74912CD8CF10E0D9
:10335000B3CFBE016F5F7F4FCE0188960E940125DB
:1033600047ED56E0BE01685D7F4F89ED96E00E9413
:10337000EE45CE0188960E94C42460E176E0CE013D
:1033800001960E94962484EF482E55245394612C74
:10339000712CC301B2010E941A7464ED76E0C6017B
:1033A0000E94E1342BEAE22E22E1F22E02EB12E13E
:1033B0009E012F5F3F4F48EE53E060E070E0C60192
:1033C0000E94E24A6AE775E0CE0188960E940A25CB
:1033D000BE01685D7F4FCE0101960E940723892BB5
:1033E00029F011E08D819E81089708F410E0CE014C
:1033F00088960E94C424111117C060E176E0CE01C6
:1034000001960E949624E4EF4E0EE1E05E1E611CE0
:10341000711CF0E74F16F7E15F066104710409F0D3
:10342000B8CF80EA96E064CF9924939421962FAD8B
:103430002197213009F0912C86E896E00E94AF2870
:103440005ACF892DC05CDF4F0FB6F894DEBF0FBE98
:10345000CDBFDF91CF911F910F91FF90EF90DF9043
:10346000CF90BF90AF909F908F907F906F905F9024
:103470004F903F902F900895BF92CF92DF92EF929E
:10348000FF920F931F93CF93DF93EC018C01085BA6
:103490001F4FF801808186FF76C07496B08061E08E
:1034A00070E080E090E00E941A748B2D0E940374FB
:1034B0006C01990FEE08FF0860E08B2D0E94987355
:1034C000C114D104E104F10421F4C12CD12C760102
:1034D000C394C701B6010E9462899B01AC0160E000
:1034E00070E080E894E40E94BC8B20E030E040E88B
:1034F0005FE30E944F8B9B01AC01FE01ED59FF4F32
:1035000060817181828193810E94BC8BFE01E559AB
:10351000FF4F20813181428153810E94C3899B01E9
:10352000AC0160E074E284E799E40E94BC8B6B011B
:103530007C01FE01E35AFF4F0190F081E02D3097AE
:1035400049F120E030E048EC51E4608171818281F2
:1035500093810E944F8BFE01E959FF4F20813181F9
:10356000428153810E94C38920E030E040E85FE35C
:103570000E94508B9B01AC01C701B6010E94BC8B1D
:103580006B017C0107C0C12C8CE3D82E8CE1E82EA6
:1035900086ECF82EA701960160E0CE010E9404504F
:1035A000CC5BDF4F188219821A821B82F80180815E
:1035B0008F79808381E0DF91CF911F910F91FF90F0
:1035C000EF90DF90CF90BF9008950C94CA830C9435
:1035D000CA830C94CA830C94CA83AF92BF92CF92D1
:1035E000DF92EF92FF920F931F93CF93DF9300D060
:1035F000CDB7DEB78C015C018FEBA80EB11CF501D5
:10360000E080F18062E875E0C7010E94228E892B7C
:1036100039F067E875E0C7010E94228E892BA9F472
:10362000F801EF53FF4F80810E940374BC01990F92
:10363000880B990B0E9464892DE332E64BE95BE32A
:103640000E94C3896B017C0107C0C12C8CE3D82E7A
:103650008CE1E82E86ECF82EF501A080B1806CE8B4
:1036600075E0C5010E94228E892B39F061E574E076
:10367000C5010E94228E892BA1F4F801EF53FF4F60
:1036800080810E940374BC01990F880B990B0E94E2
:1036900064892FE037E648E75CE30E94C3896B0149
:1036A0007C01A701960160E0C8010E94045080914E
:1036B000A7149091A814009711F48BEA94E1BE012D
:1036C0006F5F7F4F681B790B072E000C880B990BDF
:1036D0000E9464899B01AC0161E0C8010E94045012
:1036E000F801EE53FF4F608171816F5F7F4F7183EF
:1036F0006083072E000C880B990B0E9464899B0144
:10370000AC0162E0C8010E940450F801EC5BFF4F7D
:103710001082118212821382349680818F79808385
:1037200081E00F900F90DF91CF911F910F91FF904B
:10373000EF90DF90CF90BF90AF900895CF92DF923F
:10374000EF92FF921F93CF93DF93EC0181E10E94F0
:10375000D86F182F82E10E94D86F682F70E086E042
:10376000759567958A95E1F7072E000C880B990BE4
:1037700017FF19C00E94648920E030E040E85EE352
:103780000E94C3896B017C01612F619570E080E02C
:1037900090E00E9464899B01AC01C701B6010E94C0
:1037A000508B905816C00E94648920E030E040E8B9
:1037B0005EE30E94C3896B017C01612F70E080E0B1
:1037C00090E00E9464899B01AC01C701B6010E9490
:1037D000508B9B01AC0160E0CE010E940450FE01C1
:1037E000EC5BFF4F1082118212821382C85BDF4FA5
:1037F00088818F79888381E0DF91CF911F91FF903D
:10380000EF90DF90CF900895CF930E94FA4CC82F8D
:10381000882369F08EE00E94D86F682F60628EE086
:103820000E94766F8EE00E94D86F85FDFBCF8C2FB3
:10383000CF910895CF93DF93EC010E944046CE01D3
:10384000DF91CF910C94CE4D80E00895AF92BF925E
:10385000CF92DF92FF920F931F93CF93DF93EC01F0
:103860005B018A0181EF98EDFA0191838083FB016E
:1038700091838083CE01C2960E940C43F82EC82EFD
:10388000880FDD08C65ADF4FCE010E942C0B88231B
:1038900019F0CE010E944011F501D182C082CD28DD
:1038A000B1F06F2DFF0C770B880B990B0E94648988
:1038B0002BEE32EE4EEC5FE30E94C38929E23CE935
:1038C00046E353E40E94508B0E942E8C02C060E0BD
:1038D00070E0F8017183608381E0DF91CF911F91E7
:1038E0000F91FF90DF90CF90BF90AF900895089513
:1038F000089508950895CF93DF93EB01BC0180EC08
:1039000098E00E946C2660E280EC98E00E94F3252B
:10391000BE0180EC98E0DF91CF910C94E125CF932C
:10392000C62FBC0180EC98E00E946C2660E280EC1F
:1039300098E00E94F3256C2F80EC98E0CF910C94D6
:10394000136CCF93DF93EC0160E474E00E940A25CE
:10395000CE01DF91CF9108953F924F925F926F9287
:103960007F928F929F92AF92BF92CF92DF92EF920F
:10397000FF920F931F93CF93DF93CDB7DEB7AB9733
:103980000FB6F894DEBF0FBECDBF7C018B011A824B
:103990001982FE01339683E2DF011D928A95E9F7D1
:1039A000DB01ED91FC910088F189E02D40E550E0CC
:1039B00061E975E0C8010995892B09F4CAC164EA77
:1039C00075E08DE990E10E942B8E6AEA75E08DE941
:1039D00090E10E940C8E6CEB75E08DE990E10E9405
:1039E0000C8E0E94C9284C9724F460E0C8010E9404
:1039F000CB4366EC75E08DE990E10E940C8E61E9A5
:103A000075E08DE990E10E940C8E0E94C9288F9785
:103A100024F460E0C8010E94CB436FEC75E08DE9AF
:103A200090E10E940C8EF701608571858DE990E12F
:103A30000E940C8E0E94C9284A9724F460E0C801B5
:103A40000E94CB4369ED75E08DE990E10E940C8EF8
:103A5000B12C73E6C72ED12CD7011296ED91FC91B3
:103A600013970584F685E02D8281B81670F58B2CAE
:103A7000912CC401880F991F0190F081E02DE80F6F
:103A8000F91F60817181CE0186960E9415428AA538
:103A90009BA58796C80ED91ECE0186960E94C42487
:103AA000BFEF8B1A9B0AD7011296ED91FC911397E9
:103AB0000584F685E02D828190E08816990619F03C
:103AC000BFEFCB1ADB0AB394C7CF4AE0BE016F5FEA
:103AD0007F4FC60101960E94CE86BE016F5F7F4F69
:103AE0008DE990E10E940C8E0E94C9288A9724F4E7
:103AF00060E0C8010E94CB436CEE75E08DE990E177
:103B00000E940C8E0E94C928459724F460E0C801E9
:103B10000E94CB4361E176E08DE990E10E940C8E3A
:103B20000E94C928849724F460E0C8010E94CB4316
:103B3000D7011296ED91FC911397638574858DE9F9
:103B400090E10E940C8E0E94C9288A9724F460E0BC
:103B5000C8010E94CB4367E276E08DE990E10E94C4
:103B60000C8E40918B1350918C1360918D1370913A
:103B70008E13CE0186960E94395D45E250E0BE016B
:103B80006F5F7F4FCE0186960E94554ACE01869682
:103B90000E94C424BE016F5F7F4F8DE990E10E94B7
:103BA0000C8EEDE9F0E1DF010D900020E9F71197AF
:103BB00082E28C9301900020E9F731978CE28083B8
:103BC000B12C9DE9C92E90E1D92E22E2A22E3AE332
:103BD000532E4DE7442E5CE2352ED7011296ED911F
:103BE000FC9113970584F685E02D8281B81608F0C4
:103BF0008AC00E94C9288F9724F460E0C8010E94FF
:103C0000CB43F60101900020E9F73197A0828B2C7D
:103C1000912C3401660C771CD7011296ED91FC9122
:103C200013970584F685E02D0190F081E02DE60DD7
:103C3000F71D0190F081E02D61897289CE01869691
:103C40000E940A2545E250E0BE016F5F7F4FCE0122
:103C500086960E94554ACE0186960E94C424BE01D3
:103C60006F5F7F4F8DE990E10E940C8EF60101900D
:103C70000020E9F73197A082F60101900020E9F7D2
:103C800031975082D7011296ED91FC9113970584DC
:103C9000F685E02D80819181FC01E60DF71D6081A4
:103CA0007181CE0186960E94154245E250E0BE0128
:103CB0006F5F7F4FCE0186960E94554ACE01869651
:103CC0000E94C424BE016F5F7F4F8DE990E10E9486
:103CD0000C8EBFEF8B1A9B0AD7011296ED91FC91C7
:103CE00013970584F685E02D828190E0F60101901E
:103CF0000020E9F731978816990611F0308201C04B
:103D00004082B3946ACF61E0C8010E94CB430E9415
:103D100054746B017C010E945474DC01CB018C193A
:103D20009D09AE09BF0980319742A105B105C0F4D4
:103D3000D801ED91FC910084F185E02DC801099531
:103D40000C9774F46AE070E080E090E00E941A74CE
:103D5000E2CF8EE098E00E94AF2808EF11E029C082
:103D6000FE0131967F01C12CD12CC8010E9464252F
:103D700097FD0AC0F70181937F01FFEFCF1ADF0A99
:103D80002CE0C216D10489F7D801ED91FC9104888A
:103D9000F589E02DC8010995CD28F9F28A858EA311
:103DA0008B858FA38C8588A7CE0186960E948E86F0
:103DB0008C018AEF97E00E94AF28B80180EC98E070
:103DC0000E944C6DC801AB960FB6F894DEBF0FBED3
:103DD000CDBFDF91CF911F910F91FF90EF90DF90BA
:103DE000CF90BF90AF909F908F907F906F905F909B
:103DF0004F903F900895CF93DF93EC0161E975E018
:103E00000E940A25CE01DF91CF910895CF93DF93D1
:103E1000EC0162308BE07807C1F050F4613086E04D
:103E2000780781F061307B40B1F467E476E015C03B
:103E300066308BE0780761F068307B4061F468E9B8
:103E400076E00BC067E376E008C064E676E005C084
:103E50006AE776E002C062EB76E0CE010E940A25B6
:103E6000CE01DF91CF9108952F923F924F925F92B2
:103E70006F927F928F929F92AF92BF92CF92DF927A
